:100000000C94E4030C942B040C94BF070C942B0465
:100010000C942B040C942B040C942B040C942B04A4
:100020000C942B040C942B040C942B040C947A0D3C
:100030000C942B040C948D1B0C942B040C942B040B
:100040000C942B040C942B040C942B040C94D31BB5
:100050000C942B040C942B040C942B040C942B0464
:100060000C942B040C942B040C942B040C942B0454
:100070000C942B045905C905AB05ED0501060706CF
:100080000B060F06130617061B061E06220626067B
:100090004D0E6F0E5D0F6F0E5D0FB40ED70E5D0F20
:1000A0002C0F3F0F3712371264126412BF12DB1489
:1000B000DB14DB14FB12DB14F613F613B114DB14A0
:1000C000DB14C7148042803E3C3A3B456843413FC5
:1000D0003D2B3567697A790078141E806A801D1679
:1000E000041A1F806B061B07082120806C2C19093D
:1000F000171522806D11050B0A1C23806E80100DD0
:10010000182425806F360E0C122726807037380F82
:1001100033132D80717534802F2E8072397D2830F5
:10012000803180738064808076802A778059745C07
:100130005F66808062635A5D5E60295344575B56F8
:100140005561478080808040808080808080808072
:1001500080808080807E80807C80808080808080A5
:100160008080807B800180038080807F8080808091
:100170008080806580800280808080808080808018
:10018000808080808080808080808080808054809B
:100190008080808080808080808080808080588087
:1001A000808080808080808080808080804D8050B2
:1001B0004A808080494C51804F52808080804E80A0
:1001C000464B48800A0025303862003A200025302E
:1001D0003258000A722F63203031323334353637CB
:1001E0000A00756E65787065637465642073636179
:1001F0006E20636F64652061742045305F46303A3D
:1002000020253032580A00756E6578706563746514
:1002100064207363616E20636F646520617420469F
:10022000303A20253032580A00756E657870656363
:10023000746564207363616E20636F64652061740C
:100240002046303A20463028636C65617220616E2A
:100250006420636F6E742E290A00756E6578706570
:1002600063746564207363616E20636F64652061ED
:10027000742045303A20253032580A00756E657872
:10028000706563746564207363616E20636F646579
:1002900020617420494E49543A20253032580A00D2
:1002A0004F76657272756E0A0025690D0A007062DC
:1002B00075663A2066756C6C0A004B6579626F61F1
:1002C00072642073746172742E0A00555342206365
:1002D0006F6E666967757265642E0A000D0A696E35
:1002E00069740A003003500053002F0032002000D0
:1002F0006B006500790062006F00610072006400AD
:10030000200063006F006E007600650072007400CC
:100310006500720000000E0374002E006D002E00B8
:100320006B002E000000040309040902740004019C
:1003300000A032090400000103010100092111019C
:1003400000012240000705810308000A090401009A
:1003500001030000000921110100012236000705F8
:10036000820308000A0904020002030000000921B8
:100370001101000122220007058303200001070567
:100380000303200001090403000103000000092108
:100390001101000122390007058403200001120128
:1003A000100100000008EDFE1265010001020001CD
:1003B00005010906A101050719E029E71500250136
:1003C0009508750181020508190129059505750132
:1003D00091029501750391010507190029F7150090
:1003E000250195F875018102C00631FF0974A1014C
:1003F0000975150026FF00952075088102097615FC
:100400000026FF00952075089102C005010980A112
:1004100001850216810026B7001A81002AB70075EF
:100420001095018100C0050C0901A1018503160189
:1004300000269C021A01002A9C0275109501810079
:10044000C005010906A101050719E029E7150025E6
:10045000019508750181029501750881010508194A
:100460000129059505750191029501750391010515
:1004700007190029FF150026FF0095067508810061
:10048000C00A002530325820006B6579626F6172B6
:10049000645F7265706F72743A20004C45443A2074
:1004A000253032580A0064656C5F6B65795F62695C
:1004B000743A2063616E27742064656C3A2025309D
:1004C00032580A006164645F6B65795F6269743AEF
:1004D0002063616E2774206164643A2025303258AD
:1004E0000A003F00433E20004C25640A000A092D03
:1004F00020436F6E736F6C65202D0A4553432F7137
:100500003A09717569740A000A092D204D616769FD
:1005100063202D0A643A0964656275670A783A09AE
:100520006465627567206D61747269780A6B3A0957
:100530006465627567206B6579626F6172640A6DCC
:100540003A096465627567206D6F7573650A763A5E
:100550000976657273696F6E0A733A097374617410
:1005600075730A633A09636F6E736F6C65206D6F04
:1005700064650A302D343A096C61796572302D3426
:10058000284631302D4634290A506175733A096284
:100590006F6F746C6F616465720A6E3A094E4B52EC
:1005A0004F0A003F004E4B524F3A206F66660A00DA
:1005B0004E4B524F3A206F6E0A0074696D65725F40
:1005C00072656164333228293A202530346C580A28
:1005D000006B6579626F6172645F6E6B726F3A2057
:1005E00025580A006B6579626F6172645F69646C9B
:1005F000653A2025580A006B6579626F6172645F05
:1006000070726F746F636F6C3A2025580A00686FC0
:1006100073745F6B6579626F6172645F6C6564733C
:1006200028293A2025580A000A092D20537461749C
:100630007573202D0A004743433A20342E392E3259
:10064000204156522D4C4942433A20312E382E300B
:1006500073766E204156525F415243483A2061768C
:100660007233350A004F5054494F4E533A204C557F
:1006700046412045585452414B455920434F4E5313
:100680004F4C4520434F4D4D414E44204E4B524F11
:10069000204B45594D41505F53454354494F4E20DF
:1006A000343039360A004255494C443A20633236D8
:1006B00039326165202831363A30373A3039204FA7
:1006C00063742020342032303136290A00564944E0
:1006D0003A2030784645454428742E6D2E6B2E29DD
:1006E000205049443A203078363531322850532F43
:1006F00032206B6579626F61726420636F6E76651C
:100700007274657229205645523A20307830303064
:10071000310A00444553433A20636F6E7665727424
:100720002050532F32206B6579626F6172642074A0
:100730006F205553420A000A092D205665727369CD
:100740006F6E202D0A000A6D6F7573653A206F6613
:10075000660A000A6D6F7573653A206F6E0A000AAB
:100760006B6579626F6172643A206F66660A000A8F
:100770006B6579626F6172643A206F6E0A000A6D70
:1007800061747269783A206F66660A000A6D617456
:100790007269783A206F6E0A000A64656275673A7A
:1007A000206F6E0A000A64656275673A206F66669C
:1007B0000A000A0A626F6F746C6F616465722E2E94
:1007C0002E2000433E20000011241FBECFEFD4E0B6
:1007D000DEBFCDBF04B603FE27C0809166029091B4
:1007E0006702A0916802B09169028730904BA740E0
:1007F000B04BD1F410926602109267021092680218
:100800001092690214BE84B7877F84BF0FB6F89434
:10081000A8958091600088618093600010926000CC
:100820000FBEE0E0F8E3099511E0A0E0B1E0E6E1F9
:10083000F2E402C005900D92A233B107D9F722E08D
:10084000A2E3B1E001C01D92A636B207E1F70E9413
:10085000BF0A0C9409210C940000FF93EF93E091E0
:100860003201F0913301309709F00995EF91FF9132
:100870000895FC018591803011F0EFDFFBCF0895E2
:10088000FF27E0E230E247FF0CC0419597FF09C027
:10089000EDE26095709580959095611D711D811DAB
:1008A000911D27FF02C0219530E350E2AA27660F71
:1008B000771F881F991FAA1FA41710F0A41B639508
:1008C0005A95A9F7AA3008F0A95FA05DAF93F395F8
:1008D000611571058105910541F7ED3211F4EF9332
:1008E000F395F21718F43F93F395FBCF8F91B5DF93
:1008F000FA95E1F70895E991F9918591803021F019
:10090000853219F0AADFF9CF089520E0E8945591D7
:100910005532C1F3503311F4689455915A3348F469
:10092000505390F3220F022E220F220F200D250F7D
:10093000F4CF0EF4219589919991533619F35337D9
:1009400029F1533559F1BC0188279927E8945C3681
:1009500021F48991999168945591543639F446EF70
:100960007EF077FF0DC08FEF9FEF0AC055374AE04A
:1009700039F0583540E121F0523642E009F008954F
:10098000FF93EF937DDFEF91FF91B7CFFF93EF934D
:10099000FC0181918030B9F360DFFBCFFF93EF93CF
:1009A00068DFF1CFDF93CF93CDB7DEB72596A3DF16
:1009B000CF91DF910895E82FE695E695E695F0E072
:1009C000EA5CFE4F4081282F277081E090E002C052
:1009D000880F991F2A95E2F7242F30E02823392326
:1009E000232B29F4842B808381E0809335010895A3
:1009F000E82FE695E695E695F0E0EA5CFE4F20816B
:100A0000382F377081E090E002C0880F991F3A9527
:100A1000E2F7422F50E048235923452B31F08095CF
:100A20008223808381E0809335010895E6E3F1E03D
:100A300080E28E0F11928E13FDCF089580914D02AA
:100A4000816080934D020E94CE06E6E3F1E080E2F1
:100A50008E0F11928E13FDCF0895CF931092350112
:100A60008091550186FF03C08EEF0E94F8040E941A
:100A7000A707C82F882361F01F928F9389EA92E01D
:100A80009F938F930E94D2040F900F900F900F901E
:100A9000809158018111E1C0E09134018E2F90E0E6
:100AA0008E30910508F0D7C0FC01E65CFF4F0C9436
:100AB0002B1ECA3A31F178F4C338F9F0C438F9F092
:100AC000C11134C00E9416050E94F81480EA92E019
:100AD0000E943904C0C0C13E71F020F4C03E31F51F
:100AE00082E092C0C03F29F0CC3F01F582E191E065
:100AF0000AC081E089C084E087C083E8AAC08CEF87
:100B0000A8C08FE091E09F938F9385E191E09F9340
:100B10008F930E94311E0E94950F0E947C061092B6
:100B200034010F900F900F900F9097C0C7FD02C037
:100B30008C2F8FC00E9416050E94F8141F92CF932D
:100B40008CE792E09F938F930E94D2040F900F90B6
:100B50000F900F9080C0C93509F47DC020F4C231D8
:100B600009F479C008C0CE3721F0C03F21F483E0FA
:100B70004BC08BE049C0C7FD03C08C2F806869C0A3
:100B80000E9416050E94F8141F92CF938AE592E006
:100B9000D9CFC43831F0C03F31F0C33889F483E88D
:100BA00024C08CEF22C00E9416050E94F81489E22E
:100BB00092E09F938F930E94D2040F900F904DC0AC
:100BC000C7FD02C08C2F11C00E9416050E94F814A8
:100BD0001F92CF9387E092E0B5CFC231E1F1C935E2
:100BE000D1F1C7FD05C08C2F80680E94F80433C086
:100BF0000E9416050E94F8141F92CF9382EE91E096
:100C0000A1CFC43141F585E08093340126C0C737B8
:100C100011F586E0F9CFC13EF1F487E0F5CFC03F92
:100C2000D1F488E0F1CFC431B1F489E0EDCFC03F19
:100C300091F48AE0E9CFC73771F40AC0C03E59F495
:100C40008CE0E2CFC03F39F48DE0DECFCE3719F42F
:100C50008EEF0E94DB041092340181E0CF91089561
:100C6000E82FF0E0EA5CFE4F80810895CF92DF929A
:100C7000EF92FF920F931F93CF93DF9383ED91E059
:100C80000E94390486E3E82E81E0F82EC0E0D0E02F
:100C90009EECC92E91E0D92E06EC11E0DF93CF93A4
:100CA000DF92CF920E94D2048BEC91E00E94390433
:100CB000F70181917F010E94401B1F928F931F9328
:100CC0000F930E94D20484EC91E00E943904219693
:100CD0008DB79EB708960FB6F8949EBF0FBE8DBF16
:100CE000C032D105D9F6DF91CF911F910F91FF90BE
:100CF000EF90DF90CF900895982F82FB882780F99E
:100D000090FD826091FD84600C9452084FB7F89476
:100D10002091590130915A0180915B0190915C01C1
:100D20008217930781F0F901EE0FFF1FE35AFE4F80
:100D3000808191812F5F3F4F2F71332730935A016C
:100D40002093590102C080E090E04FBF0895CF93F7
:100D5000DF93EC010E946108882341F0209731F075
:100D600085E08A95F1F700002197F4CFCE01DF915D
:100D7000CF910895CF93DF93C2E3D0E00E94610842
:100D8000811108C0209731F085E08A95F1F70000C5
:100D90002197F4CFCE01DF91CF9108950E945E0894
:100DA0000E946E08E9E6F0E0808188608083E99A1D
:100DB00008958AE1815019F40E94860608959FB72C
:100DC000F89440915B0150915C0120915901309160
:100DD0005A019FBF4217530779F7EFE9FFE03197B8
:100DE000F1F700C00000E6CFEF92FF920F931F9340
:100DF000CF93DF93E82E10925801E9980E945B0888
:100E00000E946E088FE891E00197F1F700C00000A2
:100E10000E946B080E945E0880E197E20E94A7068C
:100E2000892B11F48AE077C0C0E0D0E011E0F12C0A
:100E300001E090E59A95F1F7C7010C2E02C0959557
:100E400087950A94E2F780FF04C010270E946E087D
:100E500002C00E946B080E94BA06892B11F482E03E
:100E60005AC082E390E00E94A706892B11F483E028
:100E700052C02196C830D105E1F680E58A95F1F798
:100E8000112319F00E946E0802C00E946B080E9494
:100E9000BA06892B11F484E03EC082E390E00E9400
:100EA000A706892B11F485E036C090E59A95F1F7F5
:100EB0000E946E08C2E3D0E00E947108882341F0CE
:100EC000209741F025E02A95F1F700002197F4CF13
:100ED000CD2B11F486E01FC082E390E00E94A706AC
:100EE000892B11F487E017C00E94BA06892B11F4F0
:100EF00088E011C0C2E3D0E00E947108811108C0EF
:100F0000209741F085E08A95F1F700002197F4CF12
:100F1000CD2B81F489E0809358010E945E080E94E5
:100F20006E08E99A80E0DF91CF911F910F91FF90B9
:100F3000EF9008950E945E080E946E08E99ADF9182
:100F4000CF911F910F91FF90EF900C94D9064FB75E
:100F5000F89420915B0130915C018091590190914E
:100F60005A014FBF2817390729F0109258010E94E3
:100F70008606089580E28093580180E008951F92CC
:100F80000F920FB60F9211242F933F934F935F93BD
:100F90006F937F938F939F93AF93BF93CF93EF9371
:100FA000FF930E94610881116BC0809157018F5F90
:100FB000809357018A3028F4823068F4813031F010
:100FC00054C08A30D9F08B3029F14FC00E9471088B
:100FD00081114BC055C08091560186958093560172
:100FE0000E947108882309F44BC0809156018068E3
:100FF00080935601809100018F5F40C00E9471086C
:1010000090910001882319F090FF2FC039C090FD06
:101010002CC036C00E947108882339F140915601D6
:1010200050E0CFB7F89480915B0190915C019C01F6
:101030002F5F3F4F2F7133276091590170915A01F3
:101040002617370761F0880F991FFC01E35AFE4FFE
:101050005183408330935C0120935B0104C08EEA8E
:1010600092E00E943904CFBF04C080915701809361
:101070005801109257011092560181E080930001AF
:10108000FF91EF91CF91BF91AF919F918F917F9100
:101090006F915F914F913F912F910F900FBE0F90E5
:1010A0001F901895CF93C82F8DEE0E94F4068C2FB9
:1010B000CF910C94F4065998519A08955198599AE1
:1010C00008955198599A85E08A95F1F7000089B101
:1010D0008695817008955898509A08955098589A16
:1010E00008955098589A85E08A95F1F7000089B1E3
:1010F000817008958091C101089508959FB7F89473
:101100001092A0019FBF90915702943009F057C0F0
:101110009091E9009F703091EC00232F217030FDF9
:1011200020E8922B23E02093E9002091EB0020FFA0
:1011300043C02091EE0027FF3FC020919D01222354
:1011400021F02091E80025FF37C010929D0126E094
:101150003091E80035FD15C030915702343061F50B
:101160003091EB0035FD28C0215021F481E08093BF
:101170009D0122C0EFE9FFE03197F1F700C00000C8
:10118000E7CF8093F1008091E80085FD0AC080914F
:10119000E80080FFFCCF8091E8008E778093E80024
:1011A00006C08FB7F89421E02093A0018FBF9F70F5
:1011B0009093E90080E008959F709093E9008FEF8D
:1011C0000895CF93DF9300D01F92CDB7DEB7209163
:1011D0005702243021F523E029839B838A8382E010
:1011E0008093E9008FEF9091E800815095FD06C053
:1011F00095ED9A95F1F700008111F5CF8091E80007
:1012000085FF0DC040E050E063E070E0CE01019644
:101210000E94860B8091E8008E778093E8000F9003
:101220000F900F90DF91CF910895CF93DF9300D06F
:101230001F92CDB7DEB79C0180915702843019F51B
:1012400092E099833B832A839093E9008FEF9091FA
:10125000E800815095FD06C095ED9A95F1F70000E4
:101260008111F5CF8091E80085FF0DC040E050E08E
:1012700063E070E0CE0101960E94860B8091E80049
:101280008E778093E8000F900F900F90DF91CF91B1
:101290000895CF93DF93EC0190915702943009F0B9
:1012A00046C080910B018823D9F080910C018823DE
:1012B000B9F09093E9008FEF9091E800815095FD8F
:1012C00006C095E19A95F1F700008111F5CF809164
:1012D000E80085FF2CC040E050E060E270E017C0FD
:1012E00081E08093E9008FEF9091E800815095FDB7
:1012F00006C095ED9A95F1F700008111F5CF809128
:10130000E80085FF14C040E050E068E070E0CE01E6
:101310000E94860B8091E8008E778093E80080E23F
:10132000FE01A1EAB1E001900D928A95E1F7DF910B
:10133000CF910895089520919E012F5F822F62E33F
:101340000E941F1E992319F020939E010895109268
:101350009E018091A001882371F180915702843011
:1013600041F58091E9008F702091EC00922F9170EF
:1013700020FD90E8892B93E09093E9009091EB0099
:1013800090FF14C09091EE0097FF10C09091E8007C
:1013900095FF03C01092F100F9CF9091E80090FF03
:1013A00005C09091E8009E779093E8008F7080933D
:1013B000E9001092A001089542E061EC81E00E94F2
:1013C000910C42E061EC82E00E94910C42E261ECFF
:1013D00083E00E94910C42E261EC84E00C94910C59
:1013E00080915902833009F455C030F4813071F096
:1013F000823009F48EC008958A3009F47AC08B30A7
:1014000009F460C0893009F09CC020C08091580266
:10141000813A09F096C08091E800877F8093E800C8
:1014200080915C0290915D02892B21F460E281EA57
:1014300091E003C060E080E090E070E00E94D30B98
:101440008091E8008B778093E8000895809158029E
:10145000813209F076C080915C0290915D02009724
:1014600019F0039709F06DC08091E800877F8093A1
:10147000E8008091E80082FD05C08091570281114B
:10148000F8CF5FC08091F1008093C1018091E800A6
:101490008B7753C080915802813A09F052C08091F5
:1014A0005C0290915D02892B09F04BC08091E800AD
:1014B000877F8093E8008091E80080FFFCCF8091D7
:1014C0000B0136C0809158028132D9F580915C02BF
:1014D00090915D02892BA9F58091E800877F809328
:1014E000E8000E94C60C80915A0280930B010C9474
:1014F000F81480915802813221F58091E800877FAD
:101500008093E8000E94C60C80915B028093C20128
:10151000089580915802813AA1F48091E800877F74
:101520008093E8008091E80080FFFCCF8091C201A9
:101530008093F1008091E8008E778093E8000C940E
:10154000C60C0895089508958091C10180939F016C
:101550001092C10180E00E947C060E941E050C943E
:10156000F8140C94A40A0E94661B809155028823EB
:1015700029F00E94751B81110C94700B089584B79B
:10158000877F84BF0FB6F894A8958091600088612A
:1015900080936000109260000FBE90E080E80FB66C
:1015A000F89480936100909361000FBE8EE798E0FD
:1015B0000E943B1B8CED92E00E9439040E94A20A1B
:1015C0000E9417100E94170D0E946A0D8091E20080
:1015D00084608093E200789480915702843019F0FF
:1015E0000E94750FF9CF8BEC92E00E9439040E94A3
:1015F000191081E091E00E94900F8AEB92E00E9426
:1016000039040E94A30A80915702853019F40E9480
:10161000B30AF9CF0E941D100E94750FF4CF0E94EB
:10162000891B80919F018093C10108950C940F0B39
:10163000292F332723303105C9F064F421303105D7
:1016400081F02230310509F043C084E790E02AE2BE
:1016500033E042C021323105F1F02232310541F14F
:1016600037C082E190E02EE933E036C0992781301F
:10167000910541F08230910541F0892B49F5E6E270
:10168000F3E005C0E6E1F3E002C0E4EEF2E08491AD
:1016900090E09F0121C06430D8F4E62FF0E0EE0F17
:1016A000FF1FE75DFE4F2081318189E090E014C08B
:1016B000643070F470E0FB01EE0FFF1FEF5DFE4F32
:1016C00020813181FB01E35EFE4F808190E004C008
:1016D00080E090E020E030E0FA013183208308953B
:1016E00084E089BD86E089BD09B400FEFDCF80910C
:1016F000D8008F7D8093D8008091E0008260809335
:10170000E0008091E00081FDFCCF0895CF92DF9250
:10171000EF92FF920F931F93CF93DF93EC018B0116
:101720007A010E94E50C811135C0E114F10439F011
:10173000F70180819181081B190BC80FD91FC12C9B
:10174000D12C0115110529F18091E80085FD18C003
:101750008091E8008E778093E8000E94750FE11475
:10176000F10449F0F70180819181C80ED91ED18220
:10177000C08285E00FC00E94E50C882311F30AC0E7
:1017800089918093F10001501109FFEFCF1ADF0A10
:10179000D8CF80E0DF91CF911F910F91FF90EF9014
:1017A000DF90CF90089520915E0230915F0226175E
:1017B000370748F06115710539F42091E8002E775C
:1017C0002093E80001C0B90140E06115710591F175
:1017D00020915702222309F440C0253009F43FC06C
:1017E0002091E80023FD3DC02091E80022FD2FC09C
:1017F0002091E80020FFE9CF2091F20030E0FC01C9
:10180000CF016115710559F02830310540F48191FF
:101810008093F100615071092F5F3F4FF1CF41E09C
:101820002830310509F040E02091E8002E77209320
:10183000E800CBCF4111CCCF0AC08091570288235A
:1018400061F0853061F08091E80083FD0AC08091ED
:10185000E80082FFF2CF80E0089582E0089583E0FF
:10186000089581E0089520915E0230915F0226176D
:10187000370748F06115710539F42091E8002E779B
:101880002093E80001C0B901FC0120E06115710559
:1018900079F180915702882309F43DC0853009F41D
:1018A0003CC08091E80083FD3AC08091E80082FD51
:1018B0002CC08091E80080FFE9CF8091F20090E099
:1018C0006115710559F08830910540F424912093F9
:1018D000F1003196615071090196F2CF21E008972D
:1018E00009F020E08091E8008E778093E800CECF69
:1018F0002111CFCF0AC080915702882361F0853033
:1019000061F08091E80083FD0AC08091E80082FFC9
:10191000F2CF80E0089582E0089583E0089581E0A9
:101920000895982F953058F59093E900981739F05D
:101930007091EC002091ED005091F00003C0242F35
:10194000762F50E021FF19C03091EB003E7F30939D
:10195000EB003091ED003D7F3093ED003091EB00D6
:1019600031603093EB007093EC002093ED005093C6
:10197000F0002091EE0027FF07C09F5FD3CF8F704C
:101980008093E90081E0089580E0089580915802F5
:1019900087FF11C08091E80082FD05C08091570249
:1019A0008111F8CF11C08091E8008B770BC0809136
:1019B0005702882349F08091E80080FFF8CF80919A
:1019C000E8008E778093E80008952091E40030913C
:1019D000E50095E64091EC00842F817040FF22C025
:1019E0008091E80080FD1CC080915702882391F00F
:1019F000853091F08091EB0085FD10C04091E400AE
:101A00005091E5004217530729F39A01915011F7BD
:101A100084E0089582E0089583E0089581E00895C8
:101A200080E008954091E80042FFDECF08950E94D3
:101A3000740D0E94770DE0EEF0E08081816080837C
:101A4000E8EDF0E080818F77808319BCE3E6F0E079
:101A50008081816080831092560208950E94740DE7
:101A60000E94770D8091D8008F778093D800809165
:101A7000D80080688093D8008091D8008F7D8093B3
:101A8000D80084E089BD86E089BD09B400FEFDCFA1
:101A90001092570210925302109255021092540263
:101AA00042E060E080E00E94910C8091E1008E7F36
:101AB0008093E1008091E20081608093E200809158
:101AC000E20088608093E2008091E0008E7F809346
:101AD000E0000895E3E6F0E080818E7F808381E07E
:101AE000809356020C942E0D1092E20008951092ED
:101AF000E10008951F920F920FB60F9211242F93B9
:101B00003F934F935F936F937F938F939F93AF9385
:101B1000BF93EF93FF938091E10082FF0BC0809110
:101B2000E20082FF07C08091E1008B7F8093E1009B
:101B30000E949B098091E10080FF19C08091E20022
:101B400080FF15C08091E2008E7F8093E20080913B
:101B5000E20080618093E2008091D80080628093EF
:101B6000D80019BC85E0809357020E94B10A809189
:101B7000E10084FF30C08091E20084FF2CC084E04B
:101B800089BD86E089BD09B400FEFDCF8091D800F3
:101B90008F7D8093D8008091E1008F7E8093E1005B
:101BA0008091E2008F7E8093E2008091E20081606C
:101BB0008093E20080915302882311F084E007C0F3
:101BC0008091E30087FD02C081E001C083E0809343
:101BD00057020E94160B8091E10083FF24C0809180
:101BE000E20083FF20C08091E100877F8093E100C5
:101BF00082E080935702109253028091E1008E7F21
:101C00008093E1008091E2008E7F8093E2008091DA
:101C1000E20080618093E20042E060E080E00E94A8
:101C2000910C0E949A09FF91EF91BF91AF919F9102
:101C30008F917F916F915F914F913F912F910F9075
:101C40000FBE0F901F9018951F93CF93DF93CDB7C2
:101C5000DEB7AA970FB6F894DEBF0FBECDBFE8E59A
:101C6000F2E088E08E0F9091F10091938E13FBCFFC
:101C70000E94F0098091E80083FF1FC18091580203
:101C800090915902492F50E04A30510508F015C192
:101C9000FA01E85BFF4F0C942B1E803881F08238EC
:101CA00009F00BC180915C028F708093E9008091F4
:101CB000EB0085FB882780F91092E90006C080912F
:101CC000540290915502911182609091E800977FA3
:101CD0009093E8008093F1001092F100C8C0282F83
:101CE0002D7F09F0EAC0882319F0823061F0E5C049
:101CF00080915A02813009F0E0C0933009F080E011
:101D0000809355022BC080915A02811127C0809187
:101D10005C028F7009F4D1C08093E9002091EB0040
:101D200020FF1CC0933021F48091EB00806214C02E
:101D30009091EB0090619093EB0021E030E0A901DD
:101D400002C0440F551F8A95E2F74093EA001092B3
:101D5000EA008091EB0088608093EB001092E9002C
:101D60008091E800877F86C08111A7C010915A0238
:101D70001F778091E3008078812B8093E30080912E
:101D8000E800877F8093E8000E94C60C8091E800FD
:101D900080FFFCCF8091E30080688093E300111105
:101DA00002C082E001C083E08093570286C0805861
:101DB000823008F082C080915A0290915B028C3D83
:101DC00053E0950779F583E08A838AE289834FB7E8
:101DD000F894DE01139620E03EE051E2E32FF0E0BC
:101DE00050935700E49120FF03C0E295EF703F5FEE
:101DF000EF708E2F90E0EA3010F0C79601C0C096C9
:101E00008D939D932F5F243149F74FBF8091E80058
:101E1000877F8093E8006AE270E0CE0101960E941D
:101E2000D30B14C0AE014F5F5F4F60915C020E9404
:101E3000180BBC01892B09F440C09091E800977FF2
:101E40009093E80089819A810E94330C8091E80088
:101E50008B778093E80031C0803879F58091E80075
:101E6000877F8093E800809153028093F1008091F6
:101E7000E8008E778093E8000E94C60C1EC0811196
:101E80001CC090915A029230C0F48091E800877F84
:101E90008093E800909353020E94C60C80915302F5
:101EA000811106C08091E30087FD02C081E001C07E
:101EB00084E0809357020E94DC098091E80083FF50
:101EC0000AC08091E800877F8093E8008091EB0052
:101ED00080628093EB00AA960FB6F894DEBF0FBE27
:101EE000CDBFDF91CF911F910895CF93809157027D
:101EF0008823A1F0C091E900CF709091EC00892F68
:101F0000817090FD80E8C82B1092E9008091E80074
:101F100083FD0E94240ECF70C093E900CF910895F5
:101F20009093C8018093C7010895E091C701F09193
:101F3000C801309721F00190F081E02D099480E0F4
:101F40000895EF92FF920F931F93CF93DF93E09149
:101F5000C701F091C8013097B1F18C010280F38183
:101F6000E02D099580914D0282FF2DC080FF04C0B5
:101F700089E894E00E943904E80110E283E8E82E41
:101F800084E0F82E80914D0280FF0BC088811F9263
:101F90008F93FF92EF920E94D2040F900F900F90B8
:101FA0000F90115021961111EDCF80914D0280FFBD
:101FB0000AC081E894E0DF91CF911F910F91FF90CB
:101FC000EF900C943904DF91CF911F910F91FF9006
:101FD000EF9008952091C5013091C60182179307B3
:101FE00071F09093C6018093C501E091C701F09113
:101FF000C801309721F00680F781E02D09940895FB
:102000002091C3013091C4018217930771F090931E
:10201000C4018093C301E091C701F091C8013097DA
:1020200021F00084F185E02D0994089508950C9421
:1020300016100E94B21B0C941E05CF92DF92EF92F5
:10204000FF920F931F93CF93DF9300D000D000D067
:10205000CDB7DEB70E942D058AECC82E81E0D82EC0
:1020600000E010E0E02E802F0E943006F601419142
:102070006F01F42EF826B1F40F5F1F4F00321105E7
:1020800089F78FEF89838A831B820E94BB1B816043
:10209000782F9D838C8349815A816B818D810E9429
:1020A000DA1047C090914D0291FF04C08E830E94C8
:1020B00036068E8120E030E04F2D50E0922FBA019D
:1020C000022E02C0759567950A94E2F760FF2BC057
:1020D0002983EA8221E030E0690102C0CC0CDD1CDA
:1020E0009A95E2F790E08C219D21892B09F420E05C
:1020F0002B830E94BB1B8160782F9D838C83498139
:102100005A816B818D810E94DA1049815A816B81DD
:102110007C818D810E94531BF801E653FE4F808124
:10212000C826C08206C02F5F3F4F2830310531F6E8
:10213000A3CF0E94521B1091C9010E94950F18173E
:1021400041F10E94950F8093C90190914D0292FF39
:102150000EC090FF0CC01F928F938BE994E09F9369
:102160008F930E94D2040F900F900F900F90809148
:10217000C90126960FB6F894DEBF0FBECDBFDF9122
:10218000CF911F910F91FF90EF90DF90CF900C9423
:10219000641B26960FB6F894DEBF0FBECDBFDF914D
:1021A000CF911F910F91FF90EF90DF90CF90089506
:1021B0000C947C06CF93DF93CDB7DEB72B970FB689
:1021C000F894DEBF0FBECDBF942F4F83252F5887C5
:1021D00069877A878B874A855B85452B21F02F3F5E
:1021E00009F59F3FF9F4DE01119686E0FD01119299
:1021F0008A95E9F785E0FE01379601900D928A9560
:10220000E1F749815A816B817C818D819E810E9499
:10221000A1172B960FB6F894DEBF0FBECDBFDF918E
:10222000CF9108954F81588569857A858B850E9465
:10223000531BD9CFCF93882309F4A4C0C82F8CEFA8
:102240008C0F813A48F48C2F0E94BF1D81119AC0D7
:102250008C2F0E94301A0CC080E28C0F883058F40A
:10226000C77081E001C0880FCA95EAF70E94DB1AA7
:10227000CF910C94151B8BE58C0F833078F4C53A05
:1022800029F0C63A31F083E890E005C081E890E09B
:1022900002C082E890E0CF910C94EA0F88E58C0FA1
:1022A000853108F06FC0C83A61F1C93A69F1CA3A9C
:1022B00071F1CB3A79F1CC3A81F1CD3A89F1CE3A4C
:1022C00091F1CF3A99F1C13BA1F1C03BA9F1C23BD9
:1022D000B1F1C33BB9F1C43BC1F1C53BC9F1C63B48
:1022E000D1F1C73BD9F1C83BE1F1C93BE9F1CA3BA8
:1022F000F1F1CB3BF9F1CC3B09F43FC080E090E039
:102300003EC082EE90E03BC089EE90E038C08AEE9D
:1023100090E035C085EB90E032C086EB90E02FC0B6
:1023200083EB90E02CC084EB90E029C087EB90E039
:1023300026C08CEC90E023C08DEC90E020C083E8B8
:1023400091E01DC08AE891E01AC082E991E017C0CF
:1023500084E991E014C081E292E011C083E292E04E
:102360000EC084E292E00BC085E292E008C086E2F3
:1023700092E005C087E292E002C08AE292E0CF914B
:102380000C940010CF910895882329F19CEF980FA9
:10239000913A18F40E94831A0DC090E2980F983079
:1023A00058F4877091E001C0990F8A95EAF7892F58
:1023B0000E94E11A0C94151B9BE5980F933020F4B2
:1023C00080E090E00C94EA0F885A853120F480E098
:1023D00090E00C9400100895882321F00E94DB1AED
:1023E0000C94151B0895882321F00E94E11A0C9487
:1023F000151B0895CF92DF92EF92FF920F931F93D8
:10240000CF93DF9300D000D000D0CDB7DEB725E06A
:10241000FC01DE01119601900D922A95E1F7FC0175
:1024200040813181F280258122952F7063817481F2
:10243000672B09F4C0C23F3F19F44F3F09F4BBC2F8
:102440006C0149833A8389819A812E830E94EF1916
:10245000182F092F0E94EE190E94FE18E02FE29516
:10246000EF70F0E0EE5AFF4F2E810C942B1E802F60
:10247000807F902F9F70092F882311F00295007F95
:10248000FF2049F0002309F447C2802F0E94EE1A72
:102490000E94151B41C2812F0E94C411002309F420
:1024A0008AC2802F0E94F41A26960FB6F894DEBFD7
:1024B0000FBECDBFDF91CF911F910F91FF90EF9095
:1024C000DF90CF900C94151B802F807F902F9F70F2
:1024D000092F803211F00295007F112319F011307D
:1024E00001F129C0FF20A9F0802F222349F12130DA
:1024F00039F526960FB6F894DEBF0FBECDBFDF913B
:10250000CF911F910F91FF90EF90DF90CF900C949F
:10251000FE1A222319F0213009F44DC20E94011B3A
:102520002CC0FF20E9F0263008F045C20E94D81ADE
:10253000802329F022C0FF20F1F0211115C0802F47
:1025400026960FB6F894DEBF0FBECDBFDF91CF91B8
:102550001F910F91FF90EF90DF90CF900C94EC11B2
:10256000253008F028C209C0F601858180FFD4C15A
:102570008F708583E4CF2111E3C1802F51C1202FBB
:1025800026952695237030E02115310521F0213064
:102590003105C9F010C2FF2021F0812F902F9370D8
:1025A00002C080E090E026960FB6F894DEBF0FBE22
:1025B000CDBFDF91CF911F910F91FF90EF90DF90F2
:1025C000CF900C94EA0FFF2021F0812F902F937071
:1025D00002C080E090E026960FB6F894DEBF0FBEF2
:1025E000CDBFDF91CF911F910F91FF90EF90DF90C2
:1025F000CF900C940010802F837009F078C0F110F8
:10260000DAC1812F829586958770880F880F912F68
:102610009F70C92ED12CE12CF12C082E04C0CC0CBB
:10262000DD1CEE1CFF1C0A94D2F714FF12C04FE011
:1026300050E060E070E004C0440F551F661F771F34
:102640008A95D2F7CB01BA016095709580959095E7
:1026500003C060E070E0CB01202F26952695237003
:10266000422F50E042305105D1F04330510559F12D
:102670006C297D298E299F294130510541F12696EB
:102680000FB6F894DEBF0FBECDBFDF91CF911F9183
:102690000F91FF90EF90DF90CF900C9413196C295D
:1026A0007D298E299F2926960FB6F894DEBF0FBE8E
:1026B000CDBFDF91CF911F910F91FF90EF90DF90F1
:1026C000CF900C9425190E941319C701B6012696C4
:1026D0000FB6F894DEBF0FBECDBFDF91CF911F9133
:1026E0000F91FF90EF90DF90CF900C940119FF2095
:1026F00019F0802F817001C08695882309F45BC191
:10270000812F829586958770880F880F912F9F70F3
:10271000C92ED12CE12CF12C082E04C0CC0CDD1CD0
:10272000EE1CFF1C0A94D2F714FF12C04FE050E0D9
:1027300060E070E004C0440F551F661F771F8A9544
:10274000D2F7CB01BA01609570958095909503C042
:1027500060E070E0CB01202F269526952370422F54
:1027600050E042305105D1F04330510559F16C2908
:102770007D298E299F294130510541F126960FB6BA
:10278000F894DEBF0FBECDBFDF91CF911F910F91A7
:10279000FF90EF90DF90CF900C94CA196C297D299F
:1027A0008E299F2926960FB6F894DEBF0FBECDBFA7
:1027B000DF91CF911F910F91FF90EF90DF90CF901D
:1027C0000C94DC190E94CA19C701B60126960FB6EF
:1027D000F894DEBF0FBECDBFDF91CF911F910F9157
:1027E000FF90EF90DF90CF900C94B819103F41F11B
:1027F00018F4103E48F48BC0123F09F450C0D8F1D1
:10280000133F09F460C083C01F70802F8F71FF20B9
:1028100021F00E945119812F93CE0E947219812FAD
:1028200026960FB6F894DEBF0FBECDBFDF91CF91D5
:102830001F910F91FF90EF90DF90CF900C94F311C8
:10284000FF20A9F0253008F0B6C0802F8F712696A2
:102850000FB6F894DEBF0FBECDBFDF91CF911F91B1
:102860000F91FF90EF90DF90CF900C949719263046
:1028700008F0A1C0EACFFF20A1F0802F8F7126962B
:102880000FB6F894DEBF0FBECDBFDF91CF911F9181
:102890000F91FF90EF90DF90CF900C945119FF2093
:1028A00061F3802F8F7126960FB6F894DEBF0FBEAE
:1028B000CDBFDF91CF911F910F91FF90EF90DF90EF
:1028C000CF900C947219FF2091F0802F8F71269673
:1028D0000FB6F894DEBF0FBECDBFDF91CF911F9131
:1028E0000F91FF90EF90DF90CF900C943C192696BB
:1028F0000FB6F894DEBF0FBECDBFDF91CF911F9111
:102900000F91FF90EF90DF90CF900C943719FF203C
:10291000A1F0222309F4B1CF812F26960FB6F894A7
:10292000DEBF0FBECDBFDF91CF911F910F91FF9002
:10293000EF90DF90CF900C941A11222309F4B1CFBD
:10294000812F26960FB6F894DEBF0FBECDBFDF9164
:10295000CF911F910F91FF90EF90DF90CF900C944B
:10296000C411402F4F70612FC6010E945A1C269639
:102970000FB6F894DEBF0FBECDBFDF91CF911F9190
:102980000F91FF90EF90DF90CF900C944918402F5B
:102990004F70612FC60126960FB6F894DEBF0FBEAA
:1029A000CDBFDF91CF911F910F91FF90EF90DF90FE
:1029B000CF900C945D1C26960FB6F894DEBF0FBE28
:1029C000CDBFDF91CF911F910F91FF90EF90DF90DE
:1029D000CF9008950E94FB1A0E94CA1A0E94151BEC
:1029E00080E090E00E94EA0F80E090E00C940010FC
:1029F0000E94EB1A0C94EA140E94EF19292F2295D9
:102A00002F7030E02C3031054CF42A3031056CF455
:102A1000225031092230310588F407C02C303105AD
:102A200049F02F30310531F009C0803E48F0803F39
:102A300029F406C093FB882780F9089580E0089563
:102A400081E00895CF93DF9300D000D01F92CDB7DF
:102A5000DEB70F900F900F900F900F90DF91CF91F6
:102A60000895CF93DF9300D000D000D0CDB7DEB76C
:102A700026960FB6F894DEBF0FBECDBFDF91CF9183
:102A80000895CF93DF93C091EA018091EB01C817BD
:102A9000A1F0D0E0CE0166E070E00E940E1EFC01C5
:102AA000E451FE4F4081518162817381848195811F
:102AB0000E9431152196C770E8CFDF91CF9108951C
:102AC00040911C0250911D0260911E0270911F02E4
:102AD00080912002909121020C943115CF93DF93C5
:102AE0008091210282958F7009F05CC080911E0256
:102AF000882309F457C02091EA01D091EB0140915D
:102B00001C02C0911D02E0911F02F09120022D17BE
:102B100009F448C030E0309709F440C0CF3F11F4C9
:102B20004F3FE1F1C90166E070E00E940E1EDC013A
:102B3000A451BE4F11968C911197C8132FC08C9140
:102B400048132CC012968C911297811127C01396AE
:102B50008D919C9114978E179F0708F401978E1BF7
:102B60009F0B883C9105D0F4809121028F70806189
:102B700080932102C90166E070E00E940E1EFC01F4
:102B8000EF50FE4F90819F70906190838CE192E0B6
:102B90000E94FA11DF91CF910C9441152F5F3F4FA6
:102BA0002770B5CFDF91CF910895BF92CF92DF927A
:102BB000EF92FF920F931F93CF93DF93CDB7DEB7C2
:102BC00061970FB6F894DEBF0FBECDBF8C0185E0D4
:102BD000F801DE011D9601900D928A95E1F7D8016A
:102BE0004C9111962C9111971296EC901297139686
:102BF000CD90DC90149750911C0260911D02809141
:102C00001F0290912002009709F46EC16F3F19F4E2
:102C10005F3F09F469C1B0901E02BB2009F4C3C034
:102C200030912102C816D90628F0F601E81BF90BED
:102C3000CF0104C0809590958C0D9D1DFF24F394C9
:102C4000883C910588F0F12C307F09F0CBC07C2DB9
:102C5000D98AC88A522F6E2D89890E9422158CE14B
:102C600092E00E94FA11B4C0832F807F09F049C01E
:102C7000621314C0541312C0E11010C03F703061D1
:102C8000309321020E9460158CE192E00E94FA11BB
:102C900080912102D80115968C9331C0CD2831F155
:102CA0002F3F11F44F3F11F1FE2CE1101FC0E091B6
:102CB000EA013091EB01E31709F45CC0F0E0CF01C9
:102CC00066E070E00E940E1EDC01A451BE4F11961A
:102CD0008C911197281307C08C91481304C0129649
:102CE0008C91811103C03196E770E5CFFE2CEE2068
:102CF00009F416C180912102816080932102F12C98
:102D00000FC1621308C0541306C0E11004C08091C3
:102D10002102D801C1C04D872E878D859E850E94D6
:102D2000FC148823E1F1EE20D1F120912102822FC1
:102D300082958F7090E0029774F080911C029091C0
:102D40001D0298878F831986DB86CA862C87CE0161
:102D500007960E94FA1186E0F801ACE1B2E001901A
:102D60000D928A95E1F70E946E150E946015FF246E
:102D7000F394D6C04D872E878D859E850E94EF19CE
:102D8000292F22952F7030E0223031050CF0BCC085
:102D90009F7009F0B6C0805E883008F4C1C0C801D9
:102DA0000E94FA11E4CFC816D90608F453C0F60100
:102DB000E81BF90BCF01883C910508F450C0F12CB9
:102DC0007C2DD98AC88A522F6E2D89890E9422159E
:102DD000ECE1F2E086E0DF011D928A95E9F70E94BE
:102DE00060159EC0621314C0541312C0E11010C0CD
:102DF00080912102F8018583C8010E94FA1186E0C2
:102E0000ECE1F2E0DF011D928A95E9F7FB2C88C026
:102E10004D872E878D859E850E94FC14882309F49A
:102E2000BECFEE2009F4BBCF20912102822F8295E4
:102E30008F7090E002970CF48ECF80911C029091DD
:102E40001D029A8389831B82DD82CC822E83CE0170
:102E500001967FCF809590958C0D9D1DACCFFE2C5B
:102E6000EE2009F49CCF62132EC054132CC0209185
:102E7000210220FD1FC0822F82958F70D9F0D801CA
:102E800015962C9315978F3049F08F5F982F929558
:102E9000907F822F8F70892B15968C93C8010E948A
:102EA000FA1186E0F801ACE1B2E001900D928A954A
:102EB000E1F795CF86E0F801ACE1B2E001900D9228
:102EC0008A95E1F72DC04D872E878D859E850E94BE
:102ED000FC14811140CF80912102816080932102F6
:102EE000C8010E94FA111CC0EE2009F458CF4D878A
:102EF0002E878D859E850E94FC14882309F44FCF70
:102F00002ACF811148CF0CC0243031050CF047CFB7
:102F10009F7009F440CFF8019581907F09F03BCF75
:102F20008F2D61960FB6F894DEBF0FBECDBFDF9137
:102F3000CF911F910F91FF90EF90DF90CF90BF90B6
:102F40000895CF93DF93CDB7DEB72C970FB6F894E3
:102F5000DEBF0FBECDBF4F83588769877A878B87C7
:102F60009C87CE0107960E94D515882371F08F812A
:102F700098852A853B85232B09F43FC09F3F09F0A4
:102F800068C08F3F09F065C038C086E0FE01379603
:102F9000DE01119601900D928A95E1F76F81788597
:102FA000EA85FB85309749F17F3F11F46F3F29F1A6
:102FB0008091EB0190E09C012F5F3F4F27703327FA
:102FC0004091EA0150E02417350709F44BC06983AA
:102FD0007A83FD83EC8366E070E00E940E1EDC01C4
:102FE000A451BE4F96E0FE01319601900D929A9544
:102FF000E1F72093EB010E9441158091EA01909145
:10300000EB018917E9F190E066E070E00E940E1E86
:1030100084519E4F0E94D515882391F18091EA0139
:1030200090E066E070E00E940E1EFC01E451FE4F4D
:103030004081518162817381848195810E94311523
:103040008091EA0190E00196877099278093EA01C8
:10305000D4CF4F81588569857A858B859C850E9460
:103060003115CBCF0E94F8141092EB011092EA01B7
:10307000ECE1F2E086E0DF011D928A95E9F7BDCF31
:103080002C960FB6F894DEBF0FBECDBFDF91CF9167
:103090000895DF92EF92FF920F931F93CF93DF93E8
:1030A000FC01892B09F48AC0E12CF12CDD24D39496
:1030B000EF0121968491853709F461C058F4843773
:1030C00008F04EC0843008F06AC08130D1F0823000
:1030D00071F174C0883709F45DC050F4863709F483
:1030E00055C0873709F06AC08E2D0E94E81A54C077
:1030F0009CE7980F903708F061C08F770E94C41149
:1031000050C08F010E5F1F4FFE01849190E2980F17
:10311000983050F48770FD2D01C0FF0F8A95EAF7B3
:103120008F2F0E94EE1A14C00E941A1113C08F0133
:103130000E5F1F4FFE01C49180E28C0F883060F457
:10314000C7708D2D01C0880FCA95EAF70E94F41A46
:103150000E94151BE80125C08C2F0E94C411FACFD4
:103160009F012E5F3F4FFE01C491CC2369F08FE990
:103170009FE00197F1F700C00000C150F6CF9F011A
:103180002E5F3F4FFE01F490E9010BC00E94D81A58
:10319000E82E07C00E94EB1A0E94151B02C00E9475
:1031A0001A118F2D882341F0EFE9FFE03197F1F7F5
:1031B00000C000008150F6CFFE017ACFDF91CF91A1
:1031C0001F910F91FF90EF90DF900895609326027A
:1031D0007093270280932802909329020E94621B19
:1031E0000C94EA14609322027093230280932402C9
:1031F000909325020E94631B0C94EA1408950C948A
:10320000E6180F931F930091260210912702209138
:10321000280230912902602B712B822B932B1F9156
:103220000F910C94E6180F931F93009126021091B2
:1032300027022091280230912902602371238223E2
:1032400093231F910F910C94E6180F931F930091F5
:10325000260210912702209128023091290260272E
:103260007127822793271F910F910C94E61860E035
:1032700070E0CB010C94F2180F931F9341E050E0E3
:1032800060E070E08A019B0104C0000F111F221F43
:10329000331F8A95D2F7C901B8011F910F910C9481
:1032A000F2180F931F9341E050E060E070E004C01B
:1032B000440F551F661F771F8A95D2F7809122020F
:1032C00090912302A0912402B09125028A019B01D2
:1032D000082B192B2A2B3B2BC901B8011F910F91E9
:1032E0000C94F2180F931F9341E050E060E070E0FF
:1032F00004C0440F551F661F771F8A95D2F740956B
:103300005095609570958091220290912302A09132
:103310002402B09125028A019B01082319232A2344
:103320003B23C901B8011F910F910C94F2180F9320
:103330001F9341E050E060E070E004C0440F551F6F
:10334000661F771F8A95D2F78091220290912302FF
:10335000A0912402B09125028A019B010827192718
:103360002A273B27C901B8011F910F910C94F2182D
:103370000F931F93009122021091230220912402A7
:1033800030912502602B712B822B932B1F910F9173
:103390000C94F2180F931F930091220210912302B4
:1033A00020912402309125026023712382239323EC
:1033B0001F910F910C94F2180F931F93009122020A
:1033C0001091230220912402309125026027712759
:1033D000822793271F910F910C94F2180895CF9292
:1033E000DF92EF92FF920F931F93CF93DF938C01A5
:1033F000C0902602D0902702E0902802F090290287
:103400004091220250912302609124027091250282
:10341000C42AD52AE62AF72ACFE1D0E0D701C6018F
:103420000C2E04C0B695A795979587950A94D2F768
:1034300080FF07C0B8018C2F0E942B1C81309105A2
:1034400031F4219758F7B80180E00E942B1CDF91DE
:10345000CF911F910F91FF90EF90DF90CF90089543
:1034600090910B01992321F090910C01911109C0C9
:1034700020910D0130910E01F90132969FEF40E04D
:1034800030C0982F9695969596959F31A0F4E0912F
:103490000D01F0910E01E90FF11D877021E030E080
:1034A000A90102C0440F551F8A95E2F7CA01918114
:1034B000892B8183089590914D0290FF23C01F9224
:1034C0008F9384EC94E09F938F930E94D2040F908B
:1034D0000F900F900F9008959F3F39F04F5F4E313E
:1034E00041F051915813F8CF0DC05111F7CF942FDF
:1034F000F5CF9F3F39F0F901E90FF11D97FDFA95DE
:1035000082830895089590910B01992321F0909161
:103510000C01911109C020910D0130910E01F901AA
:103520003296205E3F4F30C0982F9695969596958F
:103530009F31A8F4E0910D01F0910E01E90FF11D0A
:10354000877021E030E0A90102C0440F551F8A9521
:10355000E2F7CA0180959181892381830895909132
:103560004D0290FF16C01F928F9386EA94E09F93BE
:103570008F930E94D2040F900F900F900F90089598
:103580003196E217F30729F090819813F9CF108252
:10359000F7CF089581E090E0E0910D01F0910E01E8
:1035A000E80FF91F1082019680329105A9F708955E
:1035B00080914C02089590914C02892B80934C028B
:1035C0000895809590914C02892380934C02089530
:1035D00080934C02089510924C02089590914B02F2
:1035E000892B80934B020895809590914B028923FB
:1035F00080934B02089510924B02089580932A0203
:10360000089510922A02089580910D0190910E0163
:10361000FC0131969C01205E3F4F80E09191911119
:103620008F5FE217F307D1F70895E0910D01F09154
:103630000E0180914C028083E0910D01F0910E010A
:10364000908180914B02892B808380912A0288236C
:1036500061F0E0910D01F0910E019081892B808342
:103660000E94041B811110922A0280910D019091F9
:103670000E010C94A10F90933301809332010895B1
:103680008295982F9C7C292F26952695982F9373A9
:10369000990F990F922B892F8A7A86959575990F94
:1036A000892B08950895CF93DF9300D000D01F9207
:1036B000CDB7DEB70F900F900F900F900F90DF9166
:1036C000CF910895089508950C94D81083B7817F01
:1036D0008C6083BF83B7816083BF7894889583B7FC
:1036E0008E7F83BF089508950895CF930E94731B22
:1036F0000E942D050E94741BC0E08C2F0E94300692
:10370000811104C0CF5FC032C1F701C081E0CF9109
:1037100008950E941E050C94F8141F920F920FB684
:103720000F9211248F939F93AF93BF9380914E027A
:1037300090914F02A0915002B09151024196A11D6B
:10374000B11D80934E0290934F02A0935002B0930C
:103750005102BF91AF919F918F910F900FBE0F902B
:103760001F90189582E084BD93E095BD9AEF97BDB8
:1037700080936E0008952FB7F89480914E02909137
:103780004F02A0915002B09151022FBF08952FB760
:10379000F89460914E0270914F0280915002909186
:1037A00051022FBF08951F920F920FB60F9211244E
:1037B0008F939F93AF93BF9380914E0290914F024E
:1037C000A0915002B09151020196A11DB11D8093AC
:1037D0004E0290934F02A0935002B0935102BF91BA
:1037E000AF919F918F910F900FBE0F901F901895E2
:1037F0000E94170DF8942FEF87EA91E62150804040
:103800009040E1F700C0000087E090EBDC0180937E
:10381000660290936702A0936802B09369029CE0ED
:1038200088E10FB6F894A895809360000FBE90933E
:103830006000FFCFE92FF0E093E0EE0FFF1F9A95B5
:10384000E1F7E80FF11DEC53FF4F9491892F8F7032
:1038500092959F700895CF93C82FCB010E941A1C98
:10386000492F90E0242F30E054E0220F331F5A9567
:10387000E1F7282B392B2038310519F480E090E04E
:1038800017C0EC2FF0E023E0EE0FFF1F2A95E1F7C1
:103890004770E40FF11D34E0EE0FFF1F3A95E1F79A
:1038A000E80FF91FEE0FFF1FE050F8498591949142
:1038B000CF91089580E090E008950895CF93C82FA8
:1038C0001F928F9388EE94E09F938F930E94D2046F
:1038D00081E090E0A0E0B0E0BC01CD0104C0660F43
:1038E000771F881F991FCA95D2F70E94FF180F9063
:1038F0000F900F900F90CF910C94F814CF938732C4
:10390000A8F58E3108F02BC1803109F49FC0F8F47E
:10391000873009F464C0A8F4863009F024C180918E
:103920004D02817F8E7F80934D028DEE94E00E9448
:10393000390483EC97E00E94390481E080935202BD
:103940004CC08B30F1F18E3009F46CC00CC1863163
:1039500009F4B0C020F4813109F4EDC004C189310B
:1039600009F491C08B3109F449C0FDC0883349F195
:1039700050F4893209F4F1C0853309F4EEC087327E
:1039800009F0F1C0EAC0833409F4E7C028F48A33AF
:1039900008F4E9C08953E4C0883409F0E4C00E9407
:1039A000F81482EB97E00E9439042FEF83ED90E347
:1039B000215080409040E1F700C000000E94F81BB9
:1039C0000CC088E095E05CC089E997E00E9439046A
:1039D00080914D02816080934D02C1E0C9C0809109
:1039E0004D02C82FC17080FFEFCF85EA97E00E949B
:1039F000390480914D02817F8E7F3DC090914D02B0
:103A000091FBCC27C0F981E0C827892FC0FB81F941
:103A100080934D02CC2319F08CE897E027C08EE705
:103A200097E02EC090914D0292FBCC27C0F981E027
:103A3000C827892FC0FB82F980934D02CC2319F04F
:103A40008FE697E013C08FE597E01AC090914D0282
:103A500093FBCC27C0F981E0C827892FC0FB83F9ED
:103A600080934D02CC2351F083E597E00E94390406
:103A700080914D02816080934D027AC086E497E088
:103A80000E943904AACF87E397E00E94390483E1BA
:103A900097E00E9439048DEC96E00E94390486EA92
:103AA00096E00E94390485E696E00E94390486E398
:103AB00096E0E6CF88E296E00E9439040E94950FD6
:103AC0001F928F938EE096E09F938F930E94D20473
:103AD00080910B011F928F9387EF95E09F938F93B7
:103AE0000E94D2048091C2011F928F9384EE95E0D0
:103AF0009F938F930E94D20480910C011F928F9309
:103B000081ED95E09F938F930E94D2040E94C71B82
:103B10009F938F937F936F938AEB95E09F938F93FF
:103B20000E94D2048DB79EB746960FB6F8949EBFFA
:103B30000FBE8DBF52CF0E94F814C0910C0181E0DE
:103B4000C827C0930C01CC2329F080EB95E00E949C
:103B500039040EC085EA95E093CF80E001C08D5115
:103B60000E945E1C3ACF83EA95E00E943904C0E0CF
:103B70008C2FCF91089580E0089580E00895CF9331
:103B8000C82F80915202882319F0813049F03EC03D
:103B9000E0910D01F0910E0180818232C9F507C0DC
:103BA000E0910D01F0910E018081823261F48C2F41
:103BB0000E94BB1D811104C08C2F0E947E1C24C05A
:103BC00081E090E021C08C2F0E94BD1D81111BC09F
:103BD000C43189F018F4CB3029F010C0C93259F043
:103BE000C83361F48DEE94E00E94390484EE94E0D1
:103BF0000E94390408C0109252020CC082EE94E078
:103C00000E94390407C081E0817006C01092520200
:103C100080E002C080E0F8CFCF91089500245527BE
:103C200004C0080E591F880F991F009729F0769538
:103C30006795B8F37105B9F7802D952F0895991BF5
:103C400079E004C0991F961708F0961B881F7A9593
:103C5000C9F780950895EE0FFF1F0590F491E02DB0
:103C60000994A0E0B0E0E7E3FEE10C94E220AE01AD
:103C70004B5F5F4FFA0161917191AF0180916202D8
:103C8000909163020E94471EE2E00C94FE20ACE09B
:103C9000B0E0EDE4FEE10C94D2207C016B018A01DE
:103CA000FC0117821682838181FFBFC1CE0101967C
:103CB0004C01F7019381F60193FD859193FF81916A
:103CC0006F01882309F4ADC1853239F493FD8591E4
:103CD00093FF81916F01853229F4B70190E00E9432
:103CE0003120E7CF512C312C20E02032A0F48B3250
:103CF00069F030F4803259F0833269F420612EC0CB
:103D00008D3239F0803339F4216028C0226024607C
:103D100025C0286023C027FD29C030ED380F3A3078
:103D200088F426FF07C0852D6AE00E94C920582E1E
:103D3000530E14C0832D6AE00E94C920382E330E22
:103D400020620CC08E3221F426FD6BC1206406C0B7
:103D50008C3611F4206802C0883641F4F60193FDD8
:103D6000859193FF81916F018111BFCF982F9F7D26
:103D70009554933028F40C5F1F4FFFE3F9830DC077
:103D8000833631F0833771F0833509F05BC022C090
:103D9000F801808189830E5F1F4F44244394512C86
:103DA000540115C03801F2E06F0E711CF801A080BB
:103DB000B18026FF03C0652D70E002C06FEF7FEF7A
:103DC000C5012C870E9426202C0183012C852F778A
:103DD000222E17C03801F2E06F0E711CF801A0808E
:103DE000B18026FF03C0652D70E002C06FEF7FEF4A
:103DF000C5012C870E941B202C012C852068222EB7
:103E0000830123FC1BC0832D90E048165906B0F4B3
:103E1000B70180E290E00E9431203A94F4CFF5019E
:103E200027FC859127FE81915F01B70190E00E94F8
:103E3000312031103A94F1E04F1A510841145104E5
:103E400071F7E5C0843611F0893639F5F80127FF9E
:103E500007C060817181828193810C5F1F4F08C010
:103E600060817181072E000C880B990B0E5F1F4F2C
:103E70002F76722E97FF09C0909580957095619569
:103E80007F4F8F4F9F4F2068722E2AE030E0A401B1
:103E90000E946920A82EA81844C0853729F42F7ED7
:103EA000B22E2AE030E025C0F22FF97FBF2E8F36E8
:103EB000C1F018F4883579F0B4C0803719F088372C
:103EC00021F0AFC02F2F2061B22EB4FE0DC08B2D7C
:103ED0008460B82E09C024FF0AC09F2F9660B92EB7
:103EE00006C028E030E005C020E130E002C020E15B
:103EF00032E0F801B7FE07C0608171818281938151
:103F00000C5F1F4F06C06081718180E090E00E5F02
:103F10001F4FA4010E946920A82EA818FB2DFF772F
:103F20007F2E76FE0BC0372D3E7FA51450F474FE15
:103F30000AC072FC08C0372D3E7E05C0BA2C372D52
:103F400003C0BA2C01C0B52C34FF0DC0FE01EA0D30
:103F5000F11D8081803311F4397E09C032FF06C023
:103F6000B394B39404C0832F867809F0B39433FDDF
:103F700013C030FF06C05A2CB31418F4530C5B184E
:103F8000B32CB31468F4B70180E290E03C870E9440
:103F90003120B3943C85F5CFB31410F43B1801C025
:103FA000312C34FF12C0B70180E390E03C870E94BF
:103FB00031203C8532FF17C031FD03C088E790E017
:103FC00002C088E590E0B7010CC0832F867859F0D5
:103FD00031FF02C08BE201C080E237FD8DE2B70104
:103FE00090E00E943120A51438F4B70180E390E0FE
:103FF0000E9431205A94F7CFAA94F401EA0DF11DE2
:104000008081B70190E00E943120A110F5CF3320CC
:1040100009F44FCEB70180E290E00E9431203A943B
:10402000F6CFF7018681978102C08FEF9FEF2C9624
:10403000E2E10C94EE20FC0105906150704001100B
:10404000D8F7809590958E0F9F1F0895FC016150C1
:10405000704001900110D8F7809590958E0F9F1FAA
:1040600008950F931F93CF93DF93FB01238121FDCD
:1040700003C08FEF9FEF28C022FF16C046815781F3
:10408000248135814217530744F4A081B1819D01F9
:104090002F5F3F4F318320838C93268137812F5FA1
:1040A0003F4F3783268310C0EB01092F182F008460
:1040B000F185E02D0995892BE1F68E819F8101968E
:1040C0009F838E83812F902FDF91CF911F910F912E
:1040D0000895FA01AA27283061F1203191F1E8947E
:1040E0006F936E7F6E5F7F4F8F4F9F4FAF4FB1E0EB
:1040F00040D0B4E03ED0670F781F891F9A1FA11DE2
:10410000680F791F8A1F911DA11D6A0F711D811DE6
:10411000911DA11D22D009F468943F91062E000C38
:104120003019000C000C3019305D3193CEF6CF0100
:104130000895462F4770405D4193B3E00FD0C9F713
:10414000F6CF462F4F70405D4A3318F0495D31FD80
:104150004052419302D0A9F7EACFB4E0A6959795D3
:10416000879577956795BA95C9F7009761057105A9
:1041700008959B01AC010A2E0694579547953795F3
:104180002795BA95C9F7620F731F841F951FA01D4D
:104190000895002480FD060E660F11F08695D1F774
:1041A000802D08952F923F924F925F926F927F924F
:1041B0008F929F92AF92BF92CF92DF92EF92FF9237
:1041C0000F931F93CF93DF93CDB7DEB7CA1BDB0BE3
:1041D0000FB6F894DEBF0FBECDBF09942A88398888
:1041E00048885F846E847D848C849B84AA84B9848F
:1041F000C884DF80EE80FD800C811B81AA81B9819B
:10420000CE0FD11D0FB6F894DEBF0FBECDBFED01AE
:064210000895F894FFCFB1
:10421600017A0849097D081509E10801012B024FB9
:104226004B004E47004241542025730A0040362277
:104236003941040B04E903B0033C0355036E038EB6
:02424600030073
:106800008800EA44E944E244040005000600070069
:10681000080009000A000B000C000D000E000F001C
:1068200010001100120013001400150016001700CC
:10683000180019001A001B001C001D001E001F007C
:10684000200021002200230024002500260027002C
:10685000280029002A002B002C002D002E002F00DC
:1068600030003100000033003400350036003700BE
:10687000380039003A003B003C003D003E003F003C
:1068800040004100420043004400450046004700EC
:10689000480049004A004B004C004D004E004F009C
:1068A000500051005200530054005500560057004C
:1068B000580059005A005B005C005D005E005F00FC
:1068C00060006100620063006400F1A18500670060
:1068D000680069006A006B006C006D006E006F005C
:1068E0007000710072007300890087008A008B00BD
:1068F000E000E100E200E300E400E500E600E7007C
:106900000100010001000100EA4401000100E2442D
:106910000100010001000100460001004A004B0097
:10692000010001004700480001000100E9440100A6
:106930000100010001000100010001003A003B00DC
:106940003C003D003E003F0040004100420043004B
:10695000010035004C0039000100440045005200A0
:1069600049000100010050004F0029004D004E0079
:1069700051000100010001000100010001000100BF
:1069800001000100010001000100010001000100FF
:1069900001000100010001000100010001004D00A3
:1069A0004A004E004B0001000100010001000100FF
:1069B00001000100010001000100010001000100CF
:1069C00001000100010001000100010001000100BF
:1069D00001000100010001000100010001000100AF
:1069E0000100010001000100490001000100010057
:1069F000010001000100010001000100010001008F
:00000001FF
